:020000040000FA
:040000003CEF00F0E1
:020008004BD0DB
:0800180099D0036A026EFF0E8D
:100020000226032200D0D8A01200030E016EE70EB4
:1000300002D8F5D7016AFE0F006EE86A015AD8A00F
:1000400012000000000600D0F8D7056A046A100EFE
:10005000F36E0134043605360250045C0350055833
:1000600005E30250045E0350055AD880003601367D
:10007000F32EEFD700501200F86A4F0EAF6E240E29
:10008000AC6E900EAB6E0001C69A540E926EE00EEE
:10009000936EC00E946E070EB46E0F0EC16EA8D094
:1000A0009EAA1BD0060EAB1412E1E1CF24F0E2CFE2
:1000B00025F0262A1EEE80F02650E126000EE222D0
:1000C000AECFE7FF24C0E1FF25C0E2FF1100AE5034
:1000D000AE50AB98AB8811000AD0F2A408D0F294CD
:1000E000094A0A2A8070086AD6CF07F01100110069
:1000F0002650275C14E0272AE9CF00F0EACF01F070
:100100000EEE80F02750E926000EEA22EF50006E36
:1001100000C0E9FF01C0EAFFD880120004D0E868FF
:10012000006ED8A012001200266A276A9D8A9F8A54
:10013000F28EF28C12009D9A0EEE80F0000EEE6AA6
:10014000E82EFDD7266A276A9D8A1200F29ED8CF34
:100150005AFEE8CF5BFEE0CF5CFEE9CF5DFEEACF62
:100160005EFEE1CF5FFEE2CF60FED9CF61FEDACF67
:1001700062FEF6CF63FEF7CF64FEF5CF65FEF3CFE8
:1001800066FEF4CF67FEA6CF68FEF28E0001A19254
:10019000B90EB26EB30EB36E212A400E215C03E19C
:1001A0001D4A1E2A216AF29E5ACED8FF5BCEE8FF76
:1001B0005CCEE0FF5DCEE9FF5ECEEAFF5FCEE1FF01
:1001C00060CEE2FF61CED9FF62CEDAFF63CEF6FFEA
:1001D00064CEF7FF65CEF5FF66CEF3FF67CEF4FF82
:1001E00068CEA6FFF28E10009EA8FED7AD6E12005C
:1001F00094988B9894968B9693908A9093928A92E7
:1002000093948A9493968A9693988A98949A8B9AC0
:1002100092928992929A899A9296899694948B94C2
:100220001A6A176A226A92908980320EF6DE9290DC
:1002300089907ADF80DFCD6AF294F28A870ED56EDC
:10024000B16AA192A082B26AB36AD08EA292B10EB4
:10025000B16E4EDF0B6EC10E0B5C07E3FE0E0B5C46
:1002600002E3F7D702D00D6AF4D70BAE2DD00D6A9A
:100270008992800E0B5C06E10BC00DF00E680F68D2
:10028000898221D0900E0B5C06E10BC00DF0106846
:100290001168898218D0A00E0B5C06E10BC00DF02E
:1002A0001268136889820FD0B00E0B5C05E10BC099
:1002B0000DF01468156807D0C00E0B5C04E10BC08C
:1002C0000DF01768898254D10D5203E18992C1D78C
:1002D0004FD1800E0D5C16E10E2803E10BC00EF02D
:1002E00010D00BC00FF0010E0E5C09E18B988B96BD
:1002F0008A908A928A948A968A988B9A01D0899257
:100300000E6836D1900E0D5CD8A4CDD0102803E134
:100310000BC010F0C7D00BC011F0010E105CD8A4B8
:10032000BFD011BA828A11AA829A119A115208E199
:100330008B888B868A808A828A848A868A98AFD0C4
:10034000010E115C08E18B988B868A808A928A94D0
:100350008A968A98A4D0020E115C08E18B888B865D
:100360008A888A848A828A908A9699D0030E115C40
:1003700008E18B888B868A808A828A948A968A880A
:100380008ED0040E115C08E18B988B868A808A924D
:100390008A948A868A8883D0050E115C08E18B884E
:1003A0008B968A808A828A948A868A8878D0060E7A
:1003B000115C08E18B888B968A808A828A848A867F
:1003C0008A886DD0070E115C08E18B888B868A8045
:1003D0008A928A948A968A9862D0080E115C08E103
:1003E0008B888B868A808A828A848A868A8857D07C
:1003F000090E115C08E18B888B868A808A828A9438
:100400008A868A884CD00A0E115C08E18B888B861C
:100410008A808A928A848A868A8841D00B0E115CEF
:1004200008E18B988B968A808A828A848A868A8859
:1004300036D00C0E115C08E18B888B968A908A82EC
:100440008A848A868A982BD00D0E115C08E18B98DD
:100450008B868A808A828A848A968A8820D00E0E29
:10046000115C08E18B888B968A908A828A848A86BE
:100470008A8815D00F0E115C08E18B888B968A90C4
:100480008A928A848A868A880AD0100E115C07E1D3
:100490008B988B968A908A928A948A968A9801D0B1
:1004A0008992106865D0A00E0D5C2AE1122803E144
:1004B0000BC012F024D00BC013F0010E125C1DE132
:1004C00013B0818813A0819813B2818613A28196FC
:1004D00013B4818413A4819413B6818213A68192EC
:1004E00013B8818013A8819013BA828613AA8296CA
:1004F00013BC828813AC829801D08992126838D0DC
:10050000B00E0D5C0AE1142803E10BC014F004D016
:100510000BC015F07CEC05F02BD0C00E0D5C28E173
:100520000DC016F0172824E10BC017F0CBEC05F036
:10053000225202E18ED61CD0010E225C02E119D0BB
:1005400017D0020E225C03E138EF06F011D0030E43
:10055000225C03E1AAEF07F00BD0040E225C03E15A
:10056000E8EF08F005D0050E225CD8B448EF0AF099
:1005700070D678EC00F00B6EC10E0B5C07E3FE0E3C
:100580000B5C02E3F6D702D00D6AF3D70BAE2FD087
:100590000D6A8992800E0B5C06E10BC00DF00E68AF
:1005A0000F68898222D0900E0B5C06E10BC00DF023
:1005B00010681168898219D0A00E0B5C06E10BC08F
:1005C0000DF012681368898210D0B00E0B5C06E142
:1005D0000BC00DF014681568898207D0C00E0B5C43
:1005E00004E10BC00DF0176889827AEF05F00D5217
:1005F00003E189927AEF05F0800E0D5C18E10E2878
:1006000003E10BC00EF011D00BC00FF0010E0E5C19
:100610000AE18B988B968A908A928A948A968A9815
:100620008B9A8B9401D089920E687AEF05F0900E28
:100630000D5CD8A4FDD1102803E10BC010F0F7D158
:100640000BC011F0010E105CD8A4EFD18B988B96E3
:100650008A908A928A948A968A988B9A8B94070EAB
:10066000115C02E18B84E0D1270E115C02E18B86E4
:10067000DBD12D0E115C02E18A88D6D12E0E115CE1
:1006800002E18B8AD1D12F0E115C04E18B868A8422
:100690008A88CAD1300E115C07E18B888B868A80EC
:1006A0008A828A848A86C0D1310E115C03E18B86EE
:1006B0008A80BAD1320E115C06E18B888B868A88DB
:1006C0008A848A82B1D1330E115C06E18B888B86D5
:1006D0008A808A828A88A8D1340E115C05E18B86D3
:1006E0008A808A868A88A0D1350E115C06E18B88C3
:1006F0008A808A828A868A8897D1360E115C07E1C1
:100700008B888A808A828A848A868A888DD1370EED
:10071000115C04E18B888B868A8086D1380E115C4F
:1007200008E18B888B868A808A828A848A868A8876
:100730007BD1390E115C07E18B888B868A808A8297
:100740008A868A8871D13A0E115C07E18B888B8684
:100750008A808A848A868A8867D13B0E115C06E18A
:100760008A808A828A848A868A885ED13C0E115C5D
:1007700005E18B888A828A848A8656D13D0E115C77
:1007800006E18B868A808A828A848A884DD13E0ED1
:10079000115C06E18B888A828A848A868A8844D1A1
:1007A0003F0E115C05E18B888A848A868A883CD159
:1007B000410E115C03E0610E115C07E18B888B86B2
:1007C0008A808A828A848A882FD1420E115C03E053
:1007D000620E115C06E18A808A828A848A868A880F
:1007E00023D1430E115C03E0630E115C04E18A82A5
:1007F0008A848A8819D1440E115C03E0640E115C6E
:1008000006E18B868A808A828A848A880DD1450E89
:10081000115C03E0650E115C06E18B888A828A8494
:100820008A868A8801D1460E115C03E0660E115C4F
:1008300005E18B888A848A868A88F6D0470E115C07
:1008400003E0670E115C06E18B888A808A828A84C5
:100850008A86EAD0480E115C03E0680E115C05E15F
:100860008A808A848A868A88DFD0490E115C03E0F8
:10087000690E115C02E18A80D7D04A0E115C03E058
:100880006A0E115C04E18B868A808A82CDD04B0E81
:10089000115C03E06B0E115C04E18A848A868A880D
:1008A000C3D04C0E115C03E06C0E115C05E18A8232
:1008B0008A848A868A98B8D04D0E115C03E06D0E4A
:1008C000115C05E18B888A808A848A88ADD04E0EBF
:1008D000115C03E06E0E115C04E18A808A848A88D0
:1008E000A3D04F0E115C03E06F0E115C05E18A800E
:1008F0008A828A848A8898D0500E115C03E0700E38
:10090000115C06E18B888B868A848A868A888CD0E3
:10091000510E115C03E0710E115C06E18B888B8631
:100920008A808A868A8880D0520E115C03E0720E1B
:10093000115C03E18A848A8877D0530E115C03E04E
:10094000730E115C05E18B888A808A828A866CD05E
:10095000540E115C03E0740E115C05E18A828A84F6
:100960008A868A8861D0550E115C03E0750E115C91
:1009700004E18A808A828A8457D0560E115C03E093
:10098000760E115C05E18B868A808A848A864CD03B
:10099000570E115C03E0770E115C05E18B868A82AD
:1009A0008A868A8841D0580E115C03E0780E115C6B
:1009B00004E18B888A828A8837D0590E115C03E063
:1009C000790E115C06E18B868A808A828A868A8803
:1009D0002BD05A0E115C03E07A0E115C05E18B8876
:1009E0008B868A828A8420D05C0E115C04E18A8026
:1009F0008A868A8819D05D0E115C05E18B888B860A
:100A00008A808A8211D05E0E115C04E18B888B860D
:100A10008A860AD05F0E115C02E18A8205D07C0EC4
:100A2000115C02E18A848A8601D08992106862D0C2
:100A3000A00E0D5C2AE1122803E10BC012F024D0B5
:100A40000BC013F0010E125C1DE113B0818813A0DE
:100A5000819813B2818613A2819613B4818413A462
:100A6000819413B6818213A6819213B8818013A852
:100A7000819013BA828613AA829613BC828813AC23
:100A8000829801D08992126835D0B00E0D5C09E1D0
:100A9000142803E10BC014F003D00BC015F02CD8C0
:100AA00029D0C00E0D5C26E1172824E10BC017F0F9
:100AB00072D8225203E129EF01F01CD0010E225C12
:100AC00003E1B9EF02F016D0020E225C02E1D0D0B1
:100AD00011D0030E225C03E1AAEF07F00BD0040E45
:100AE000225C03E1E8EF08F005D0050E225CD8B4E3
:100AF00048EF0AF0B9EF02F01A0E145C07E19AD839
:100B0000020E225C02E11B6A1C6A42D01B0E145CBE
:100B100007E1020E225C03E102D01B4A1C2A38D0F6
:100B20001C0E145C10E1030E225C010ED8A4000E12
:100B3000066E040E225C010ED8A4000E061202E01E
:100B400001D0A09225D01D0E145C10E1030E225C92
:100B5000010ED8A4000E066E040E225C010ED8A46D
:100B6000000E061202E001D0A08212D0420E145CE8
:100B70000BE1155205E11B6A1C6A1A906CD803D070
:100B80001B6A1C6A1A8004D07B0E145CD8B452D83D
:100B9000899214681200175204E1166817C022F0F7
:100BA00045D0010E175C04E1166817C022F03ED054
:100BB000020E175C09E13ED816681B6A1C6A1F6AA0
:100BC000206A17C022F032D0030E175C0BE132D836
:100BD0001668216A1D6A1E6A1F6A206A8B9A17C0EE
:100BE00022F024D0040E175C15E18B888B868A8056
:100BF0008A828A848A868A98899A02D08B8A01D0CE
:100C00008B9A1668216A1D6A1E6A1F6A206A17C0BD
:100C100022F00CD0050E175C09E11668216A1D6AE6
:100C20001E6A1F6A206A8B9A17C022F00D6889928B
:100C3000176812008B988B968A908A928A948A966B
:100C40008A988B9A899A89961B6A1C6A216A1D6AFE
:100C50001E6A8B9412008B988B968A908A928A9443
:100C60008A968A988B9A8992899A89968B9412008F
:100C700078EC00F00B6EC10E0B5C07E3FE0E0B5C14
:100C800002E3F6D702D00D6AF3D70BAE2DD00D6A72
:100C90008992800E0B5C06E10BC00DF00E680F68A8
:100CA000898221D0900E0B5C06E10BC00DF010681C
:100CB0001168898218D0A00E0B5C06E10BC00DF004
:100CC0001268136889820FD0B00E0B5C05E10BC06F
:100CD0000DF01468156807D0C00E0B5C04E10BC062
:100CE0000DF0176889826CD00D5202E1899268D0AC
:100CF000800E0D5C0AE10E2803E10BC00EF004D05B
:100D00000BC00FF00E6889925BD0900E0D5C16E15F
:100D1000102803E10BC010F010D00BC011F011C06F
:100D200000F0016A0A0E026E036A25EC00F004C0AE
:100D30001BF005C01CF01068899242D0A00E0D5C1B
:100D40000AE1122803E10BC012F004D00BC013F02B
:100D50001268899235D0B00E0D5C09E1142803E1C8
:100D60000BC014F003D00BC015F0C6DE29D0C00EA6
:100D70000D5C26E10DC016F0172822E10BC017F01C
:100D80000ADF225203E129EF01F01AD0010E225CA2
:100D900003E1B9EF02F014D0020E225C02E168D741
:100DA0000FD0030E225C02E1D5D00AD0040E225CE3
:100DB00002E10ED205D0050E225CD8B448EF0AF04D
:100DC00080B4899A80A806D080B603D01B4A1C2A1A
:100DD000898601D089961BC000F01CC001F00A0E64
:100DE000026E036A25EC00F004C01FF01F50235C64
:100DF00009E01B5202E11C5203E01F52D8B4898A59
:100E00001FC023F03AD021D080A806D080B603D0EE
:100E10001B4A1C2A898601D089961BC000F01CC081
:100E200001F00A0E026E036A25EC00F004C01FF008
:100E30001F50235C09E01B5202E11C5203E01F52C9
:100E4000D8B4898A1FC023F018D017D01BC000F077
:100E50001CC001F00A0E026E036A25EC00F004C00B
:100E60001FF01F50235C09E01B5202E11C5203E0FB
:100E70001F52D8B4898A1FC023F01F5208E18B8803
:100E80008B868A808A828A848A868A9862D0010EBA
:100E90001F5C08E18B988B868A808A928A948A9656
:100EA0008A9857D0020E1F5C08E18B888B868A884F
:100EB0008A848A828A908A964CD0030E1F5C08E14D
:100EC0008B888B868A808A828A948A968A8841D087
:100ED000040E1F5C08E18B988B868A808A928A9424
:100EE0008A868A8836D0050E1F5C08E18B888B962F
:100EF0008A808A828A948A868A882BD0060E1F5C12
:100F000008E18B888B968A808A828A848A868A887E
:100F100020D0070E1F5C08E18B888B868A808A921E
:100F20008A948A968A9815D0080E1F5C08E18B88EF
:100F30008B868A808A828A848A868A880AD0090E69
:100F40001F5C07E18B888B868A808A828A948A86D6
:100F50008A888ED678EC00F00B6EC10E0B5C07E32E
:100F6000FE0E0B5C02E36AD002D00D6A67D00BAEB6
:100F700029D00D6A8072800E0B5C05E10BC00DF06C
:100F80000E680F681ED0900E0B5C05E10BC00DF0D3
:100F90001068116816D0A00E0B5C05E10BC00DF0B7
:100FA000126813680ED0B00E0B5C05E10BC00DF09B
:100FB0001468156806D0C00E0B5C03E10BC00DF081
:100FC00017683CD0A10E0D5C02E238D037D0B00ECD
:100FD0000D5C0AE1142803E10BC014F004D00BC02F
:100FE00015F07CEC05F02AD0C00E0D5C27E10DC099
:100FF00016F0172823E10BC017F0CBEC05F02252B6
:1010000003E129EF01F01AD0010E225C03E1B9EFF0
:1010100002F014D0020E225C02E12AD60FD0030E99
:10102000225C02E197D70AD0040E225C02E1D0D004
:1010300005D0050E225CD8B448EF0AF080B4899A36
:1010400080A806D080B603D01B4A1C2A898601D00E
:1010500089961BC000F01CC001F00A0E026E036AE4
:1010600025EC00F004C01FF01F50235C09E01B5268
:1010700002E11C5203E01F52D8B4898A1FC023F03A
:101080003AD021D080A806D080B603D01B4A1C2AB3
:10109000898601D089961BC000F01CC001F00A0EA1
:1010A000026E036A25EC00F004C01FF01F50235CA1
:1010B00009E01B5202E11C5203E01F52D8B4898A96
:1010C0001FC023F018D017D01DC000F01EC001F0C3
:1010D0000A0E026E036A25EC00F004C01FF01F50D8
:1010E000235C09E01D5202E11E5203E01F52D8B4F6
:1010F000898A1FC023F01F5208E18B888B868A8063
:101100008A828A848A868A9862D0010E1F5C08E1EE
:101110008B988B868A808A928A948A968A9857D0EE
:10112000020E1F5C08E18B888B868A888A848A82FB
:101130008A908A964CD0030E1F5C08E18B888B86C0
:101140008A808A828A948A968A8841D0040E1F5C9B
:1011500008E18B988B868A808A928A948A868A880C
:1011600036D0050E1F5C08E18B888B968A808A82B8
:101170008A948A868A882BD0060E1F5C08E18B88A9
:101180008B968A808A828A848A868A8820D0070EF3
:101190001F5C08E18B888B868A808A928A948A9663
:1011A0008A9815D0080E1F5C08E18B888B868A8090
:1011B0008A828A848A868A880AD0090E1F5C07E19F
:1011C0008B888B868A808A828A948A868A88C2D60D
:1011D00078EC00F00B6EC10E0B5C07E3FE0E0B5CAF
:1011E00002E36AD002D00D6A67D00BAE29D00D6A37
:1011F0008072800E0B5C05E10BC00DF00E680F686D
:101200001ED0900E0B5C05E10BC00DF0106811684C
:1012100016D0A00E0B5C05E10BC00DF01268136830
:101220000ED0B00E0B5C05E10BC00DF01468156814
:1012300006D0C00E0B5C03E10BC00DF017683CD06C
:10124000A10E0D5C02E238D037D0B00E0D5C0AE181
:10125000142803E10BC014F004D00BC015F07CEC93
:1012600005F02AD0C00E0D5C27E10DC016F017283E
:1012700023E10BC017F0CBEC05F0225203E129EF7C
:1012800001F01AD0010E225C03E1B9EF02F014D094
:10129000020E225C03E138EF06F00ED0030E225C52
:1012A00002E158D609D0040E225C02E191D704D0A5
:1012B000050E225CD8B4ECD080B4899A80A806D000
:1012C00080B603D01B4A1C2A898601D089961BC090
:1012D00000F01CC001F0060E026E036A25EC00F05F
:1012E00004C01FF01F50235C09E01B5202E11C5296
:1012F00003E01F52D8B4898A1FC023F05CD021D0EC
:1013000080A806D080B603D01B4A1C2A898601D04B
:1013100089961BC000F01CC001F00A0E026E036A21
:1013200025EC00F004C01FF01F50235C09E01B52A5
:1013300002E11C5203E01F52D8B4898A1FC023F077
:101340003AD021D080A806D080B603D01B4A1C2AF0
:10135000898601D089961BC000F01CC001F0060EE2
:10136000026E036A25EC00F004C01FF01F50235CDE
:1013700009E01B5202E11C5203E01F52D8B4898AD3
:101380001FC023F018D017D01DC000F01EC001F000
:101390000A0E026E036A25EC00F004C01FF01F5015
:1013A000235C09E01D5202E11E5203E01F52D8B433
:1013B000898A1FC023F01F5208E18B888B868A80A0
:1013C0008A828A848A868A9862D0010E1F5C08E12C
:1013D0008B988B868A808A928A948A968A9857D02C
:1013E000020E1F5C08E18B888B868A888A848A8239
:1013F0008A908A964CD0030E1F5C08E18B888B86FE
:101400008A808A828A948A968A8841D0040E1F5CD8
:1014100008E18B988B868A808A928A948A868A8849
:1014200036D0050E1F5C08E18B888B968A808A82F5
:101430008A948A868A882BD0060E1F5C08E18B88E6
:101440008B968A808A828A848A868A8820D0070E30
:101450001F5C08E18B888B868A808A928A948A96A0
:101460008A9815D0080E1F5C08E18B888B868A80CD
:101470008A828A848A868A880AD0090E1F5C07E1DC
:101480008B888B868A808A828A948A868A88A0D66C
:1014900078EC00F00B6EC10E0B5C07E3FE0E0B5CEC
:1014A00002E3F6D702D00D6AF3D70BAE2DD00D6A4A
:1014B0008992800E0B5C06E10BC00DF00E680F6880
:1014C000898221D0900E0B5C06E10BC00DF01068F4
:1014D0001168898218D0A00E0B5C06E10BC00DF0DC
:1014E0001268136889820FD0B00E0B5C05E10BC047
:1014F0000DF01468156807D0C00E0B5C04E10BC03A
:101500000DF0176889827BD1800E0D5C09E10E28F1
:1015100003E10BC00EF003D00BC00FF00E686FD1CB
:10152000900E0D5CD8A412D1102803E10BC010F06E
:101530000CD10BC011F0050E105CD8B005D18B9802
:101540008B968A908A928A948A968A988B9A929A93
:10155000899A1152D8B44DD0010E115C03E1929AD0
:10156000898A47D0020E115C04E1929A898A8A82A4
:1015700040D0030E115C04E1929A898A8A8439D0A2
:10158000040E115C05E1929A898A8A848A8831D096
:10159000050E115C05E1929A898A8A848A8629D08F
:1015A000060E115C06E1929A898A8B888A848A8663
:1015B00020D0070E115C07E1929A898A8B888B866E
:1015C0008A848A8616D0080E115C08E1929A898A6C
:1015D0008B888B868A808A848A860BD0090E115C60
:1015E00008E3929A898A8B888B868A808A848A8685
:1015F0008B8AAAD038D00A0E115C02E18A8232D0DE
:101600000B0E115C02E18A842DD00C0E115C03E1FB
:101610008A848A8827D00D0E115C03E18A848A8629
:1016200021D00E0E115C04E18B888A848A861AD040
:101630000F0E115C05E18B888B868A848A8612D016
:10164000100E115C06E18B888B868A808A848A86DC
:1016500009D0110E115C06E38B888B868A808A8400
:101660008A868B8A71D038D0120E115C02E18A8290
:1016700032D0130E115C02E18A842DD0140E115C5D
:1016800003E18A848A8827D0150E115C03E18A84DD
:101690008A8621D0160E115C04E18B888A848A86A2
:1016A0001AD0170E115C05E18B888B868A848A8696
:1016B00012D0180E115C06E18B888B868A808A8492
:1016C0008A8609D0190E115C06E38B888B868A8086
:1016D0008A848A868B8A38D037D01A0E115C02E150
:1016E0008A8232D01B0E115C02E18A842DD01C0E3E
:1016F000115C03E18A848A8827D01D0E115C03E106
:101700008A848A8621D01E0E115C04E18B888A842B
:101710008A861AD01F0E115C05E18B888B868A841D
:101720008A8612D0200E115C06E18B888B868A8017
:101730008A848A8609D0210E115C06E38B888B8609
:101740008A808A848A868B8A106859D0A00E0D5CA4
:1017500009E1122803E10BC012F003D00BC013F013
:1017600012684DD0B00E0D5C0AE1142803E10BC0E5
:1017700014F004D00BC015F07CEC05F040D0C00E86
:101780000D5C3DE10DC016F0172839E10BC017F0D4
:10179000CBEC05F0225207E1929A899A540E926E90
:1017A00029EF01F02CD0010E225C07E1929A899A70
:1017B000540E926EB9EF02F022D0020E225C07E1C5
:1017C000929A899A540E926E38EF06F018D0030E52
:1017D000225C07E1929A899A540E926EAAEF07F062
:1017E0000ED0040E225C07E1929A899A540E926EF2
:1017F000E8EF08F004D0050E225CD8B449D648D6EC
:02180000FFD710
:020000040030CA
:0300010006170ED1
:020005008580F4
:060008000FC00FE00F40E5
:00000001FF
